:020000040000FA
:0400000098EF0BF07A
:08000800056ED8CF06F0E0CF31
:1000100007F00001E9CF0DF0EACF08F0E1CF09F0D9
:10002000E2CF0AF0D9CF0BF0DACF0CF0F3CF14F017
:10003000F4CF15F0FACF16F000C00FF001C010F0A9
:1000400002C011F003C012F004C013F09DA22CEF07
:1000500000F09EB28FEF01F09DAA32EF00F09EBA41
:100060009CEF01F00FC000F010C001F011C002F0D1
:1000700012C003F013C004F00E8E0DC0E9FF08C0DB
:10008000EAFF09C0E1FF0AC0E2FF0BC0D9FF0CC0C4
:10009000DAFF14C0F3FF15C0F4FF16C0FAFF0550D5
:1000A00007C0E0FF06C0D8FF1000F2CF0EF0F29EAE
:1000B000F76AC40FF66E000EF7220900F5500EBE67
:1000C000F28E120054696D656F75743A2042656650
:1000D0006F72652077726974696E672025632025C9
:1000E00078200000F2CF0EF0F29EF76AFE0FF66E57
:1000F000000EF7220900F5500EBEF28E1200546970
:100100006D656F75743A2057616974696E67206612
:100110006F72204E44414320746F20676F206C6FD4
:1001200077207768696C652077726974696E6725D6
:100130006300F2CF0EF0F29EF76A4C0FF66E010EDE
:10014000F7220900F5500EBEF28E120054696D655B
:100150006F75743A2057616974696E6720666F72B3
:10016000204E52464420746F20676F20686967688C
:10017000207768696C652077726974696E6725639A
:100180000000F2CF0EF0F29EF76A9C0FF66E010EA1
:10019000F7220900F5500EBEF28E120054696D650B
:1001A0006F75743A2057616974696E6720666F7263
:1001B000204E44414320746F20676F206869676850
:1001C000207768696C652077726974696E6725634A
:1001D0000000F2CF0EF0F29EF76AEC0FF66E010E01
:1001E000F7220900F5500EBEF28E120054696D65BB
:1001F0006F75743A2057616974696E6720666F7213
:100200002044415620746F20676F206C6F772077F1
:1002100068696C652072656164696E6725630000BA
:10022000F2CF0EF0F29EF76A3A0FF66E020EF72248
:100230000900F5500EBEF28E120054696D656F759F
:10024000743A2057616974696E6720666F72204442
:10025000415620746F20676F20686967682077684F
:10026000696C652072656164696E67256300F2CF11
:100270000EF0F29EF76A880FF66E020EF722090062
:10028000F5500EBEF28E12005265616420657272E6
:100290006F72206F6363757265642E256300F2CF01
:1002A0000EF0F29EF76AB80FF66E020EF722090002
:1002B000F5500EBEF28E120074657374696E672578
:1002C0006300F2CF0EF0F29EF76ADC0FF66E020EBC
:1002D000F7220900F5500EBEF28E120056657273B9
:1002E000696F6E2025692E3025630000F2CF0EF075
:1002F000F29EF76A060FF66E030EF7220900F5501C
:100300000EBEF28E1200556E7265636F676E697A6B
:10031000656420636F6D6D616E642E256300010E50
:1003200001013E27D8B03F2BD8B4402BD8B4412B85
:100330009E92000132EF00F00201A2919EAAFED728
:10034000AECFA1F2A1511F0810E2A1517E080DE32A
:1003500001012851282B036A280FE96E000E0320A3
:10036000EA6EA1C2EFFF0201A281A1510A0803E0D7
:10037000A1510D08E3E19EAA0ED0036A01012851A4
:10038000280FE96E000E0320EA6E9EAAFED7AECFBC
:10039000EFFF0201F0D7A2A10AD001012851282BBA
:1003A000036A280FE96E000E0320EA6EEF6A01016E
:1003B0002851EA0801E2286B9E9A000132EF00F012
:1003C000959C8C9C959A8C9A0101375305E0959EDB
:1003D0008C8E95988C9804D0959E8C9E95988C8840
:1003E00093809382938493869388938A938C938E3D
:1003F00037530EE0929289829284928692988998DD
:10040000929A899A96908D80928096928D9208D039
:100410009282928492869288928A96809280968224
:100420000001000CCDDF929A898AEBEF0EF0020EEC
:10043000EA6E260EE96EEF500EE0050E016E006AC0
:10044000002EFED7012EFBD7F90E006E002EFED730
:100450000000EF2EF2D7000C9DC29FF29CC29EF2CC
:100460009FC203F002019EC2E9FF9FC2EAFFEF5262
:1004700006E09E2BD8B49F2B0001F2D702019C51BD
:100480009E5D006E9D519F59036E00C001F0026E8B
:100490000001000C0201A0BF10D00F0E006E9F39AA
:1004A00000160A0E005C03E2300E002602D0A051B6
:1004B000002600509EA8FED7AD6E0F0E9F170A0EA5
:1004C0009F5D02E2300E02D0A09FA0519F279F5156
:1004D0009EA8FED7AD6E0001DEEF02F0959A8C8AE1
:1004E0000201985302E092928992975309E196C2D1
:1004F0009DF295C29CF20001AFDF01C097F20201AC
:10050000959C8C8C92948984929689869288928A02
:100510000101416B406B3F6B3E6B9D82928A80BABA
:1005200003D0928880B858D041513D5D55E30BE12E
:1005300040513C5D51E307E13F513B5D4DE303E139
:100540003E513A5D49E304003D51415D44E30BE116
:100550003C51405D40E307E13B513F5D3CE303E13B
:100560003A513E5D38E3312D2ED0020195C2E9FFAC
:1005700096C2EAFFEFCF9CF295C2E9FF96C2EAFF6E
:10058000EFCF9DF29E6B9E5100018FDD02019E2BED
:10059000006E00509EA8FED7AD6E180E9E5DF3E172
:1005A0009C519EA8FED7AD6E200E9EA8FED7AD6EC4
:1005B0009DC29FF2570EA06F00016CD7200E9EA81F
:1005C000FED7AD6E0101429142950001F9DE010EA8
:1005D000016E19D10101A2D79D9202019B6B975127
:1005E0009B5DD8B0F8D0036A9B519525E96E965172
:1005F0000320EA6EEFCF9AF20101416B406B3F6B33
:100600003E6B9D82928A80AA3ED041513D5D3BE384
:100610000BE140513C5D37E307E13F513B5D33E384
:1006200003E13E513A5D2FE304003D51415D2AE371
:100630000BE13C51405D26E307E13B513F5D22E386
:1006400003E13A513E5D1EE3312D14D002019C6B53
:100650009C51000147DD02019C2B006E00509EA8BA
:10066000FED7AD6E310E9C5DF3E1010135519EA8C0
:10067000FED7AD6E429142950001A2DE010E016EE1
:10068000C2D00101BFD79D92FF0E02019A1B936A4F
:100690009AC28AFF92880101416B406B3F6B3E6BAF
:1006A0009D82928880B83ED041513D5D3BE30BE195
:1006B00040513C5D37E307E13F513B5D33E303E1EC
:1006C0003E513A5D2FE304003D51415D2AE30BE1C9
:1006D0003C51405D26E307E13B513F5D22E303E1EE
:1006E0003A513E5D1EE3312D14D002019C6B9C51AA
:1006F00000011FDD02019C2B006E00509EA8FED75A
:10070000AD6E320E9C5DF3E1010135519EA8FED71E
:10071000AD6E42914295000153DE010E016E73D021
:100720000101BFD79D92010E0201975D9B5D04E11F
:10073000995302E092948994929689960101416BB3
:10074000406B3F6B3E6B9D82928A80BA3ED0415196
:100750003D5D3BE30BE140513C5D37E307E13F5139
:100760003B5D33E303E13E513A5D2FE304003D512D
:10077000415D2AE30BE13C51405D26E307E13B513B
:100780003F5D22E303E13A513E5D1EE3312D14D07B
:1007900002019C6B9C510001F4DC02019C2B006E59
:1007A00000509EA8FED7AD6E320E9C5DF3E10101B4
:1007B00035519EA8FED7AD6E42914295000100DEF4
:1007C000010E016E20D00101BFD79D9292968986BD
:1007D00002019B2B04D7959C8C9C938093829384DD
:1007E00093869388938A938C938E985302E0929287
:1007F000898292869284929A898A92988988959A17
:100800008C9A000E016E0001000C93C296F292C207
:1008100095F294C297F2010E0201986F996B000154
:100820005DDE0150000C25C22AF196908D90C80E15
:100830000201266F0001FBDD968096928D92140EC8
:100840001E6E0201936B1E0E926F010E946F0001DB
:10085000DCDF0150000C036A01012751280F02015F
:10086000256F000E0320266F036A01012751280F10
:100870000201276F000E0320286F9D6F27C29CF294
:100880000001EADD01C028F2010E02010124016E1F
:10089000000E02200150010127272751EA0801E23A
:1008A000276B2851275D02E1276B286B020125C2C7
:1008B00001F000011AEF0FF002012B533FE027C2B5
:1008C000E9FF28C2EAFFEFCF2CF22AC203F029C2C7
:1008D000E9FF2AC2EAFFEF502C5D17E028C203F0BF
:1008E00027C2E9FF28C2EAFFEFCF2CF22AC203F0A9
:1008F00029C2E9FF2AC2EAFFEF502C5D02E2FF0E97
:1009000001D0010E016E1CD00BD028C203F027C20B
:10091000E9FF28C2EAFFEF5203E1000E016E10D09A
:1009200028C203F02751272BD8B4282B2AC203F062
:100930002951292BD8B42A2B2B07BFD7000E016EC3
:100940000001000C006A016A02012E51D8902FB1FB
:100950000026003201322FB30026003201322FB5BB
:100960000026003201322FB70026003201322FB9A3
:100970000026003201322FBB0026003201322FBD8B
:100980000026003201322FBF002600320132000162
:1009900038EF05F002012C6B2A6B0A0E2B6F296BC6
:1009A0002751281103E1000E016EC3D02C512C2BCE
:1009B000036A2725E96E28510320EA6EEFCF2DF256
:1009C0002D512D080DE1010E2A6F2C512C2B036A9D
:1009D0002725E96E28510320EA6EEFCF2DF20DD0C6
:1009E0002D512B080AE12C512C2B036A2725E96E87
:1009F00028510320EA6EEFCF2DF22D512F08D8B0E9
:100A000090D02D513908D8A08CD02D51300821E13B
:100A1000036A2C512725E96E28510320EA6EEF5016
:100A200078080AE0036A2C512725E96E2851032033
:100A3000EA6EEF5058080DE1100E2B6F2C2B2C5145
:100A40002C2B036A2725E96E28510320EA6EEFCF8D
:100A50002DF22B510A081DE12D512F0819E22D51BD
:100A6000390816E30A0E2E6F29C22FF200016AD749
:100A7000300E02012D5D0124296F2C512C2B036AAD
:100A80002725E96E28510320EA6EEFCF2DF2E4D737
:100A900048D02B51100845E12D51600806E22D5138
:100AA0007A0803E32D51DF0B01D02D512D6F2D510D
:100AB0002F0803E22D51390806E22D51400831E29A
:100AC0002D5146082EE32D512F080CE22D513908E7
:100AD00009E329392E6FF00E2E17300E2D5D2E25CD
:100AE000296F09D029392E6FF00E2E17410E2D5D7A
:100AF0000A0F2E25296F2C512C2B036A2725E96E0E
:100B000028510320EA6EEFCF2DF22D51600806E246
:100B10002D517A0803E32D51DF0B01D02D512D6F9C
:100B2000C6D72A2D04D02B510A0801E1296D29C20C
:100B300001F00001000C02012D51016A2C5D03E25D
:100B40002CC200F00CD0006A080E2E6F2C37003635
:100B50002D51005CD8B0006E01362E2FF7D7000162
:100B6000000C200E020127A9300E286F26C200F0CB
:100B700026AF07D0001E002A00C026F22D0E286FD7
:100B8000278F015026C22CF2640E2D6F0001D3DF97
:100B900000C026F2300E01240201296F26C22CF279
:100BA0000A0E2D6F0001C7DF300E002402012B6FEB
:100BB000300E01242A6F28C200F027A702D027AFE9
:100BC000279527B90BD027AF22D027B520D000C05A
:100BD00029F227B31CD000C02AF219D0300E295DAB
:100BE00016E100C029F2200E286F27A704D0279510
:100BF000278327AF2793300E2A5D09E100C02AF230
:100C0000200E296F27A7F7D7279327AF279127A56E
:100C100004D028519EA8FED7AD6E27A304D0295139
:100C20009EA8FED7AD6E27A104D02A519EA8FED75C
:100C3000AD6E2B519EA8FED7AD6E0001000C0201D7
:100C40002F6B2D6B0A0E2E6F2C6B2B6B2A6B296B67
:100C50002751281105E1006A016A026A036A3DD141
:100C60002F512F2B036A2725E96E28510320EA6EA6
:100C7000EFCF30F230512D080DE1010E2D6F2F51C5
:100C80002F2B036A2725E96E28510320EA6EEFCF48
:100C900030F20DD030512B080AE12F512F2B036A6F
:100CA0002725E96E28510320EA6EEFCF30F230514C
:100CB0002F08D8B0FAD030513908D8A0F6D030512A
:100CC000300821E1036A2F512725E96E28510320BE
:100CD000EA6EEF5078080AE0036A2F512725E96E83
:100CE00028510320EA6EEF5058080DE1100E2E6FC8
:100CF0002F2B2F512F2B036A2725E96E2851032014
:100D0000EA6EEFCF30F22E510A0844E130512F083D
:100D100040E2305139083DE3D8902935326F2A3509
:100D2000336F2B35346F2C35356F2935006E2A35EE
:100D3000016E2B35026E2C35036E003601360236FD
:100D400003360036013602360336F80E00163251ED
:100D5000002633510122345102223551032203C0AF
:100D60002CF202C02BF201C02AF200C029F2300E90
:100D7000305D2927000E2A232B232C232F512F2BC4
:100D8000036A2725E96E28510320EA6EEFCF30F27F
:100D9000BDD78BD02E511008D8A487D03051600811
:100DA00006E230517A0803E33051DF0B01D03051B5
:100DB000306F30512F0803E23051390807E23051CB
:100DC0004008D8B072D0305146086FE330512F0838
:100DD0002DE2305139082AE32935326F2A35336F35
:100DE0002B35346F2C35356F323733373437353751
:100DF000323733373437353732373337343735379F
:100E0000F00E3217300E305D3225006E000E3321A9
:100E1000016E000E3421026E000E35212C6F02C0CF
:100E20002BF201C02AF200C029F22AD02935326FF4
:100E30002A35336F2B35346F2C35356F32373337D6
:100E4000343735373237333734373537323733374E
:100E500034373537F00E3217410E305D0A0F322528
:100E6000006E000E3321016E000E3421026E000E62
:100E700035212C6F02C02BF201C02AF200C029F2EA
:100E80002F512F2B036A2725E96E28510320EA6E84
:100E9000EF50306F600806E230517A0803E33051BA
:100EA000DF0B01D03051306F84D72E510A080DE18D
:100EB0002D2D0BD0291F2A1F2B1F2C1F292BD8B4F7
:100EC0002A2BD8B42B2BD8B42C2B29C200F02AC241
:100ED00001F02BC202F02CC203F00001000C006AEA
:100EE000016A026A036A0201396B3A6B3B6B3C6B25
:100EF00038513711361135112CE0200E3D6FD89046
:100F0000313732373337343739373A373B373C3775
:100F100038513C5D08E137513B5D05E136513A5DA2
:100F200002E13551395D0FE33551395F3651D8A0B3
:100F3000363D3A5F3751D8A0373D3B5F3851D8A096
:100F4000383D3C5FD88000360136023603363D2FEF
:100F5000D6D7020EEA6E390EE96E0001000CE95098
:100F60000201296F3B0E306F9A0E2F6FCA0E2E6F43
:100F70002D6B0A0E2B6F28C234F227C233F226C221
:100F800032F225C231F230C238F22FC237F22EC20D
:100F900036F22DC235F20001A2DF0150EFCF25F26B
:100FA000ECCF26F2ECCF27F2ECCF28F2005213E17F
:100FB00002012B51010AD8A402D000010CD0295102
:100FC0000CE00F0B2B5D01E00EE229BF0CD029BD18
:100FD00004D0200E03D00201296B300E00260050F1
:100FE0009EA8FED7AD6E30C234F22FC233F22EC2AD
:100FF00032F22DC231F2386B376B366B0A0E356F19
:1010000000016DDF03C030F202C02FF201C02EF2EA
:1010100000C02DF202012B2FAED70001ECEF0FF034
:101020000201946B92988988929A899A928601011A
:10103000416B406B3F6B3E6B9D82928680A63FD09A
:1010400041513D5D3CE30BE140513C5D38E307E13C
:101050003F513B5D34E303E13E513A5D30E3040030
:101060003D51415D2BE30BE13C51405D27E307E13E
:101070003B513F5D23E303E13A513E5D1FE3312DD8
:1010800015D00201966B96510001E9EC00F00201C7
:10109000962B006E00509EA8FED7AD6E300E965D6A
:1010A000F2E1010135519EA8FED7AD6E42930001D9
:1010B000E0EC01F0FF0E016E64D00101BED79D92FD
:1010C00092988998FF0E936E81CF94F20201941B3F
:1010D0009284956B80B4952B928A0101416B406B91
:1010E0003F6B3E6B9D82928680B63FD041513D5D05
:1010F0003CE30BE140513C5D38E307E13F513B5D90
:1011000034E303E13E513A5D30E304003D51415D7B
:101110002BE30BE13C51405D27E307E13B513F5D91
:1011200023E303E13A513E5D1FE3312D15D0020167
:10113000966B9651000110EC01F00201962B006EA7
:1011400000509EA8FED7AD6E310E965DF2E1010112
:1011500035519EA8FED7AD6E42930001E0EC01F040
:10116000FF0E016E0ED00101BED79D92929A899A10
:10117000020192C2E9FF93C2EAFF94C2EFFF95C257
:1011800001F00001000C02018C6B8D6B8E6B8F9156
:10119000020E916F280E906F0101375365E05F0ECC
:1011A0001E6E02018E530FE1936B1E0E926F010EA5
:1011B000946F000105EC04F00152D8B402D0020192
:1011C00002D0000E01D0010E02018E6F3F0E1E6E86
:1011D0008E530FE1936B1E0E926F010E946F000100
:1011E00005EC04F00152D8B402D0020102D0000E86
:1011F00001D0010E02018E6F8E5303E0010E016ECD
:1012000072D1200E01012A251E6E02018E530FE1BC
:10121000936B1E0E926F010E946F000105EC04F0AB
:101220000152D8B402D0020102D0000E01D0010E4A
:1012300002018E6F8E5303E0010E016E54D1400EF9
:10124000010129251E6E0201936B1E0E926F010E85
:10125000946F000105EC04F001C08EF202018E5380
:1012600003E0010E016E3FD102018C6B020E916F03
:10127000280E906F252D7FD0020E936F260E926F51
:101280000001CEDE01C027F20201273D03D0010E8E
:10129000016E29D101012F5312E02C510201265D6C
:1012A00002E127530AE0036A8C51280FE96E020E0F
:1012B0000320EA6E26C2EFFF8C2B22D001012D51B4
:1012C0000201265D13E1275311E1010E8C5D036AD3
:1012D000280FE96E020E0320EA6E01012C51EF5C2B
:1012E00003E102018C0701010CD00201036A8C5159
:1012F000280FE96E020E0320EA6E26C2EFFF8C2B48
:10130000010102018C5164081BE18D6B8D51630852
:1013100011E391C203F090C2E9FF91C2EAFFEFCF5F
:1013200092F292519EA8FED7AD6E902BD8B4912B1D
:101330008D2BECD78C6B020E916F280E906F0400F2
:1013400027539AE18D6B0101325102018C5D8D5D55
:1013500011E291C203F090C2E9FF91C2EAFFEFCF20
:1013600092F292519EA8FED7AD6E902BD8B4912BDD
:101370008D2BE9D77ED0020E936F260E926F00015F
:101380004FDE01C027F20201273D03D0010E016E9E
:10139000AAD001012F5312E02C510201265D0BE06F
:1013A000036A8C51280FE96E020E0320EA6E26C2F2
:1013B000EFFF8C2B01D08F8121D001012D51020133
:1013C000265D12E1010E8C5D036A280FE96E020EA4
:1013D0000320EA6E01012C51EF5C04E102018C074D
:1013E0008F8101010CD00201036A8C51280FE96E34
:1013F000020E0320EA6E26C2EFFF8C2B01010201D0
:101400008C5164081BE18D6B8D51630811E391C20F
:1014100003F090C2E9FF91C2EAFFEFCF92F292513E
:101420009EA8FED7AD6E902BD8B4912B8D2BECD708
:101430008C6B020E916F280E906F04008FA19BD7CA
:101440008F918D6B0101325102018C5D8D5D11E236
:1014500091C203F090C2E9FF91C2EAFFEFCF92F28E
:1014600092519EA8FED7AD6E902BD8B4912B8D2BA8
:10147000E9D70101342D04D035519EA8FED7AD6EB9
:1014800037532EE002018E6B5F0E1E6E8E530FE1FE
:10149000936B1E0E926F010E946F000105EC04F029
:1014A0000152D8B402D0020102D0000E01D0010EC8
:1014B00002018E6F3F0E1E6E8E530FE1936B1E0E58
:1014C000926F010E946F000105EC04F00152D8B444
:1014D00002D0020102D0000E01D0010E02018E6F77
:1014E00002018EC201F00001000C0201266B5F0EAA
:1014F0001E6E26530FE1936B1E0E926F010E946FBA
:10150000000105EC04F00152D8B402D0020102D06F
:10151000000E01D0010E0201266F3F0E1E6E2653F3
:101520000FE1936B1E0E926F010E946F000105EC9C
:1015300004F00152D8B402D0020102D0000E01D052
:10154000010E0201266F200E25251E6E26530FE187
:10155000936B1E0E926F010E946F000105EC04F068
:101560000152D8B402D0020102D0000E01D0010E07
:101570000201266F26C201F00001000C9280000ECD
:1015800080B0010E016E000E01A0010E016E41EF50
:1015900017F00201286B180E1E6E28530FE1936B93
:1015A0001E0E926F010E946F000105EC04F00152C3
:1015B000D8B402D0020102D0000E01D0010E020107
:1015C000286F400E27251E6E28530FE1936B1E0EC9
:1015D000926F010E946F000105EC04F00152D8B433
:1015E00002D0020102D0000E01D0010E0201286FCC
:1015F000285301E027D0020E936F290E926F00014D
:101600000FDD01C028F20201282D01D0286B283DF2
:1016100002D0010E286F190E1E6E936B1E0E926F74
:10162000010E946F000105EC04F0020128530AE159
:1016300029519EA8FED7AD6E010135519EA8FED757
:10164000AD6E02010001000C015025C22CF2640EA7
:1016500002012D6F00019BEC05F000C025F2015046
:10166000300E08E1020126A30ED026B70CD026B911
:10167000200E04D0020126972699268101260150CA
:101680009EA8FED7AD6E25C22CF20A0E2D6F00016A
:101690009BEC05F000C025F20150300E08E102017C
:1016A00026B70BD026A109D026B9200E00010126AD
:1016B00001509EA8FED7AD6E0201300E25272551A0
:1016C0009EA8FED7AD6E0001C5EF17F026C296F2B8
:1016D00025C295F227C297F20201986B28C299F2AF
:1016E00000016EEC02F00150000C26C203F0020172
:1016F00025C2E9FF26C2EAFF2751EF5C12E026C2AD
:1017000003F025C2E9FF26C2EAFFEF5204E1000E12
:10171000016E026E0AD0252BD8B4262B0001E5D726
:10172000020125C201F026C202F0000184EF18F088
:10173000F86AD09E0D8EEA6AE96AB886090EAF6E25
:10174000000EB06EA60EAC6E900EAB6EC150C00B0C
:101750000F09C16E070EB46E186A196A0101276B72
:10176000286B010E296F0A0E2B6F2C6B2D6B2E6BC5
:10177000030E2F6F010E306F316B326B336F346F8E
:101780000D0E356F366B010E376F386F396BE80E03
:101790003A6F030E3B6F3C6B3D6B3E6B3F6B406B98
:1017A000416B429142934295436B456B280E446FC7
:1017B0002B0E466F610E476F3A0E486F496B2B0E2A
:1017C0004A6F740E4B6F3A0E4C6F4D6B2B0E4E6F73
:1017D000650E4F6F6F0E506F730E516F3A0E526F52
:1017E000536B2B0E546F650E556F6F0E566F690E4F
:1017F000576F3A0E586F596B2B0E5A6F740E5B6F02
:10180000650E5C6F730E5D6F740E5E6F5F6B2B0EFB
:10181000606F720E616F650E626F610E636F640EB2
:10182000646F656B2B0E666F670E676F650E686F72
:10183000740E696F6A6B2B0E6B6F730E6C6F740E88
:101840006D6F720E6E6F690E6F6F700E706F3A0E65
:10185000716F726B2B0E736F760E746F650E756FF2
:10186000720E766F776B2B0E786F610E796F750E37
:101870007A6F740E7B6F6F0E7C6F720E7D6F650ECC
:101880007E6F610E7F6F640E806F3A0E816F826B88
:101890002B0E836F720E846F650E856F730E866FCD
:1018A000650E876F740E886F896B2B0E8A6F640EBE
:1018B0008B6F650E8C6F620E8D6F750E8E6F670E5F
:1018C0008F6F3A0E906F916B2B0E926F936F610E2C
:1018D000946F640E956F966F720E976F986B2B0EC8
:1018E000996F9A6F610E9B6F750E9C6F740E9D6F52
:1018F0006F0E9E6F9F6B2B0EA06FA16F630EA26F7A
:101900006C0EA36F720EA46FA56B2B0EA66FA76F44
:10191000650EA86F6F0EA96F740EAA6F5F0EAB6F86
:10192000650EAC6F6E0EAD6F610EAE6F620EAF6F77
:101930006C0EB06F650EB16FB26B2B0EB36FB46FE0
:10194000650EB56F6F0EB66F740EB76F5F0EB86F22
:10195000630EB96F680EBA6F610EBB6F720EBC6F0B
:10196000BD6B2B0EBE6FBF6F690EC06F660EC16F71
:10197000630EC26FC36B2B0EC46FC56F6C0EC66F48
:10198000C76F6F0EC86FC96B2B0ECA6FCB6F6C0E13
:10199000CC6F6F0ECD6F630ECE6FCF6B2B0ED06FF3
:1019A000D16F6C0ED26F6F0ED36F6E0ED46FD56B7E
:1019B0002B0ED66FD76F6D0ED86F6F0ED96F640E6A
:1019C000DA6F650EDB6FDC6B2B0EDD6FDE6F720E78
:1019D000DF6F650EE06F610EE16F640EE26F5F0E08
:1019E000E36F740EE46F6D0EE56F6F0EE66F5F0EC2
:1019F000E76F6D0EE86F730EE96FEA6B2B0EEB6FFE
:101A0000EC6F720EED6F730EEE6F740EEF6FF06B86
:101A10002B0EF16FF26F730EF36F610EF46F760E93
:101A2000F56F650EF66F630EF76F660EF86F670E53
:101A3000F96FFA6B2B0EFB6FFC6F730EFD6F700E60
:101A4000FE6F6F0EFF6F6C0E0201006F016F026B75
:101A50002B0E036F046F730E056F720E066F710EFF
:101A6000076F086B2B0E096F0A6F730E0B6F740EE6
:101A70000C6F610E0D6F740E0E6F750E0F6F730E7F
:101A8000106F116B2B0E126F136F740E146F720E9A
:101A9000156F670E166F176B2B0E186F196F760E7A
:101AA0001A6F650E1B6F720E1C6F1D6B2B0E1E6F57
:101AB0001F6F680E206F650E216F6C0E226F700E07
:101AC000236F246B949A8B8AD180D76AD66A080ECA
:101AD0000609CA6E900ECB6EC00EF2129D92F2CF26
:101AE00025F2F29EA96AA69CA69EA680A85025BFB4
:101AF000F28EAA08D8A4A6D0F2CF25F2F29E010E4B
:101B0000A96EA69CA69EA680A85025BFF28E0101B4
:101B1000376FF2CF25F2F29E020EA96EA69CA69E0A
:101B2000A680A850020125BFF28E0101296FF2CFD5
:101B300025F2F29E030EA96EA69CA69EA680A85032
:101B4000020125BFF28E0101356FF2CF25F2F29E20
:101B5000040EA96EA69CA69EA680A850020125BFD1
:101B6000F28E0101346FF2CF25F2F29E050EA96EBE
:101B7000A69CA69EA680A850020125BFF28E010158
:101B80002F6F2F51000105E0010A0CE0030A12E05B
:101B900019D001012F6B0D0E2C6F0A0E2D6F2E6BBD
:101BA0002B6F16D0010E01012F6F0D0E2C6F2D6BB8
:101BB0002B6F0ED0020E01012F6F0A0E2C6F2D6BB2
:101BC0002B6F06D0030E01012F6F2C6B2B6B00D0F7
:101BD000F2CF25F2F29E060EA96EA69CA69EA680C6
:101BE000A850020125BFF28E0101306FF2CF25F21D
:101BF000F29E070EA96EA69CA69EA680A850020182
:101C000025BFF28E0101336FF2CF25F2F29E080E4E
:101C1000A96EA69CA69EA680A850020125BFF28EA2
:101C20000101366FF2CF25F2F29E090EA96EA69C35
:101C3000A69EA680A850020125BFF28E0101386F32
:101C4000C7D00201A96AAA0EA86EA69CA69EA68469
:101C5000F2CF00F0F29E0F01550EA76EAA0EA76EEE
:101C6000A682A6B2FED7A6940050F212010EA96E6B
:101C7000A86EA69CA69EA684F2CF00F0F29E550EFA
:101C8000A76EAA0EA76EA682A6B2FED7A694005093
:101C9000F212020EA96E010EA86EA69CA69EA68444
:101CA000F2CF00F0F29E550EA76EAA0EA76EA68286
:101CB000A6B2FED7A6940050F212030EA96E0D0E26
:101CC000A86EA69CA69EA684F2CF00F0F29E550EAA
:101CD000A76EAA0EA76EA682A6B2FED7A694005043
:101CE000F212040EA96E010EA86EA69CA69EA684F2
:101CF000F2CF00F0F29E550EA76EAA0EA76EA68236
:101D0000A6B2FED7A6940050F212050EA96E030EDD
:101D1000A86EA69CA69EA684F2CF00F0F29E550E59
:101D2000A76EAA0EA76EA682A6B2FED7A6940050F2
:101D3000F212060EA96E010EA86EA69CA69EA6849F
:101D4000F2CF00F0F29E550EA76EAA0EA76EA682E5
:101D5000A6B2FED7A6940050F212070EA96E010E8D
:101D6000A86EA69CA69EA684F2CF00F0F29E550E09
:101D7000A76EAA0EA76EA682A6B2FED7A6940050A2
:101D8000F212080EA96EA86AA69CA69EA684F2CF9F
:101D900000F0F29E550EA76EAA0EA76EA682A6B2FE
:101DA000FED7A6940050F212090EA96E010EA86E7D
:101DB000A69CA69EA684F2CF00F0F29E550EA76EBA
:101DC000AA0EA76EA682A6B2FED7A6940050F21263
:101DD000000112EF02F00101375306E00201256B0A
:101DE000000113EC04F00101949A8B9A0400640E34
:101DF0000201266F000117EC02F00400949A8B8A0E
:101E00000400640E0201266F000117EC02F00400CA
:101E10009D8A0400949A8B9A040001012751285D41
:101E2000D8B49DEF18F045C126F244C125F2000157
:101E30002BEF04F0036A01C044F1010103C045F136
:101E400045C103F044C1E9FF45C1EAFFEF502B084B
:101E5000D8A406EF18F045C128F244C127F2010EBC
:101E600002012A6F460E296F030E2B6F00015CECF6
:101E700004F0015214E1030E010144250201256F13
:101E8000000E010145210201266F286F25C227F2AD
:101E90000001CAEC04F001C029F104EF18F045C1BB
:101EA00028F244C127F2010E02012A6F920E296F17
:101EB000060E2B6F00015CEC04F001523AE1060EB5
:101EC00001014425016E000E4521036E01C0E9FFAA
:101ED000EA6EEF520EE129C126F21F0E0201276FB2
:101EE0000001B1EC05F0010135519EA8FED7AD6EA1
:101EF0001ED0060E4425016E000E4521036E01C062
:101F0000E9FFEA6EEF50200812E1070E44250201B6
:101F1000256F000E010145210201266F286F25C2A1
:101F200027F20001CAEC04F001C029F1010103EF1E
:101F300018F045C128F244C127F2010E02012A6FB0
:101F40004A0E296F030E2B6F00015CEC04F0015266
:101F50001AE1030E010144250201256F000E010163
:101F600045210201266F286F25C227F200011FECD0
:101F700006F003C03DF102C03CF101C03BF100C0DE
:101F80003AF104EF18F045C128F244C127F2010EDE
:101F900002012A6FDD0E296F0D0E2B6F00015CEC24
:101FA00004F0015245E10D0E01014425016E000EC1
:101FB0004521036E01C0E9FFEA6EEF5213E1410EC5
:101FC000E96E3DC128F23CC127F23BC126F23AC17D
:101FD00025F20001AFEF07F0010135519EA8FED7B1
:101FE000AD6E24D00D0E4425016E000E4521036E0A
:101FF00001C0E9FFEA6EEF50200818E10E0E4425FB
:102000000201256F000E010145210201266F286F94
:1020100025C227F200011FEC06F003C03DF102C00B
:102020003CF101C03BF100C03AF1010103EF18F0AF
:1020300045C128F244C127F2010E02012A6F600E49
:10204000296F050E2B6F00015CEC04F0015228E1B2
:1020500001013753D8A402D0000122D030C125F2AB
:102060000001C3EC08F0015219E00101312D15D037
:102070000201256B2551000137EC01F00201252BEF
:10208000006E00509EA8FED7AD6E130E255DF2E1E6
:10209000010135519EA8FED7AD6E000104EF18F086
:1020A000010E010144250201256F000E01014521A9
:1020B0000201266F286F25C227F2010E2A6F600EDB
:1020C000296F050E2B6F00015CEC04F001522DE12D
:1020D00001013753D8A402D0000127D0060E4425B1
:1020E000016E000E4521036E01C0E9FFEA6EEF525A
:1020F00007E10201256B0001C3EC08F013D00101D8
:10210000070E4425016E000E4521036E01C0E9FF54
:10211000EA6EEF50650807E1010E0201256F00012C
:10212000C3EC08F0010103EF18F045C128F244C1E7
:1021300027F2010E02012A6F5A0E296F050E2B6F2E
:1021400000015CEC04F0015217E10201256B2551FE
:1021500000014FEC01F00201252B006E00509EA8FB
:10216000FED7AD6E070E255DF2E1010135519EA847
:10217000FED7AD6E03EF18F045C128F244C127F237
:10218000010E02012A6F4E0E296F050E2B6F000102
:102190005CEC04F001521AE1050E01014425020134
:1021A000256F000E010145210201266F286F25C20F
:1021B00027F20001CAEC04F001C02BF12BC12CF175
:1021C00001012D6B040E2F6F03EF18F0010E0101BA
:1021D00044250201256F000E010145210201266FF1
:1021E000286F25C227F2010E2A6F4E0E296F040EAA
:1021F0002B6F00015CEC04F0015261E1050E01015E
:102200004425016E000E4521036E01C0E9FFEA6E10
:10221000EF520EE12FC126F21F0E0201276F0001BF
:10222000B1EC05F0010135519EA8FED7AD6E45D049
:10223000050E4425016E000E4521036E01C0E9FF25
:10224000EA6EEF50200839E1060E44250201256FA1
:10225000000E010145210201266F286F25C227F2D9
:102260000001CAEC04F001C02FF101012F5100015F
:1022700005E0010A0CE0030A12E019D001012F6BFE
:102280000D0E2C6F0A0E2D6F2E6B2B6F16D0010EBC
:1022900001012F6F0D0E2C6F2D6B2B6F0ED0020EC8
:1022A00001012F6F0A0E2C6F2D6B2B6F06D0030EC2
:1022B00001012F6F2C6B2B6B00D003EF18F045C181
:1022C00028F244C127F2010E02012A6F540E296F31
:1022D000050E2B6F00015CEC04F0015214E1050EB9
:1022E000010144250201256F000E01014521020173
:1022F000266F286F25C227F20001CAEC04F001C046
:1023000030F104EF18F0010E010144250201256FA0
:10231000000E010145210201266F286F25C227F218
:10232000010E2A6F540E296F040E2B6F00015CEC16
:1023300004F001523AE1050E01014425016E000E40
:102340004521036E01C0E9FFEA6EEF520EE130C194
:1023500026F21F0E0201276F0001B1EC05F001010A
:1023600035519EA8FED7AD6E1ED0050E4425016ED8
:10237000000E4521036E01C0E9FFEA6EEF50200810
:1023800012E1060E44250201256F000E01014521D0
:102390000201266F286F25C227F20001CAEC04F063
:1023A00001C030F1010103EF18F045C128F244C12A
:1023B00027F2010E02012A6F6B0E296F070E2B6F99
:1023C00000015CEC04F0015214E1070E0101442508
:1023D0000201256F000E010145210201266F286FC1
:1023E00025C227F20001CAEC04F001C032F104EF6B
:1023F00018F045C128F244C127F2010E02012A6FEC
:10240000730E296F040E2B6F00015CEC04F0015277
:102410000FE1050E0201266F1F0E276F0001B1ECC0
:1024200005F0010135519EA8FED7AD6E03EF18F0FF
:10243000010E010144250201256F000E0101452115
:102440000201266F286F25C227F2010E2A6F730E34
:10245000296F040E2B6F00015CEC04F0015226E1A1
:102460000201256B2551000161EC01F00201252BD1
:10247000006E00509EA8FED7AD6E080E255DF2E1FD
:10248000050E266F1F0E276F0001B1EC05F02E0E12
:102490009EA8FED7AD6E300E9EA8FED7AD6E010190
:1024A00035519EA8FED7AD6E03EF18F045C128F256
:1024B00044C127F2010E02012A6F660E296F040E35
:1024C0002B6F00015CEC04F0015230E10101375345
:1024D000D8A402D000012AD0050E4425016E000EBA
:1024E0004521036E01C0E9FFEA6EEF521DE143533F
:1024F0000CE129C125F2000175EC0AF00152D8B4B3
:1025000002D0010102D0000E01D0010E0101436F83
:10251000080E1E6E0201936B1E0E926F010E946FD9
:10252000000105EC04F0010103EF18F045C128F2A9
:1025300044C127F2020E02012A6F120E296F050E06
:102540002B6F00015CEC04F0015230E101013753C4
:10255000D8A402D000012AD0050E4425016E000E39
:102560004521036E01C0E9FFEA6EEF521DE14353BE
:102570000CE129C125F2000175EC0AF00152D8B432
:1025800002D0010102D0000E01D0010E0101436F03
:10259000080E1E6E0201936B1E0E926F010E946F59
:1025A000000105EC04F0010103EF18F045C128F229
:1025B00044C127F2010E02012A6F780E296F0A0E1C
:1025C0002B6F00015CEC04F0015214E10A0E0101D2
:1025D00044250201256F000E010145210201266FED
:1025E000286F25C227F20001CAEC04F001C033F1C4
:1025F00004EF18F045C128F244C127F2010E020190
:102600002A6F990E296F060E2B6F00015CEC04F007
:10261000015241E1060E01014425016E000E4521E3
:10262000036E01C0E9FFEA6EEF520EE133C126F2FC
:102630001F0E0201276F0001B1EC05F001013551B9
:102640009EA8FED7AD6E25D0060E4425016E000E65
:102650004521036E01C0E9FFEA6EEF50200819E141
:10266000070E44250201256F000E010145210201DC
:10267000266F286F25C227F20001CAEC04F001C0C2
:1026800033F10101335305E0332D01D002D0010EA7
:10269000336F03EF18F045C128F244C127F2010E51
:1026A00002012A6F830E296F060E2B6F00015CEC6E
:1026B00004F0015209E1010E0201266F000117EC3E
:1026C00002F0FF0004EF18F045C128F244C127F2E0
:1026D000010E02012A6FEB0E296F050E2B6F000110
:1026E0005CEC04F0015209E1010E0201266F0001C9
:1026F00017EC02F0FF0004EF18F045C128F244C1C6
:1027000027F2010E02012A6F8A0E296F070E2B6F26
:1027100000015CEC04F0015214E1070E01014425B4
:102720000201256F000E010145210201266F286F6D
:1027300025C227F20001CAEC04F001C031F104EF18
:1027400018F0010E010144250201256F000E010160
:1027500045210201266F286F25C227F2010E2A6F3C
:102760008A0E296F060E2B6F00015CEC04F00152FB
:1027700040E1070E01014425016E000E4521036E64
:1027800001C0E9FFEA6EEF520EE131C126F21F0EE1
:102790000201276F0001B1EC05F0010135519EA83F
:1027A000FED7AD6E24D0070E4425016E000E4521E4
:1027B000036E01C0E9FFEA6EEF50200818E1080E31
:1027C00044250201256F000E010145210201266FFB
:1027D000286F25C227F20001CAEC04F001C031F1D4
:1027E0000101315304E0312D01D001D0316B03EFF1
:1027F00018F045C128F244C127F2010E02012A6FE8
:10280000A00E296F050E2B6F00015CEC04F0015245
:1028100030E101013753D8A402D000012AD043533C
:102820000CE129C125F2000175EC0AF00152D8B47F
:1028300002D0010102D0000E01D0010E0101436F50
:10284000040E1E6E435310E10201936B1E0E926F35
:10285000010E946F000105EC04F00152D8B402D0CF
:10286000010102D0000E01D0010E0101436F03EF00
:1028700018F045C128F244C127F2010E02012A6F67
:10288000A60E296F0C0E2B6F00015CEC04F00152B8
:1028900040E10C0E01014425016E000E4521036E3E
:1028A00001C0E9FFEA6EEF520EE134C126F21F0EBD
:1028B0000201276F0001B1EC05F0010135519EA81E
:1028C000FED7AD6E25D00C0E4425016E000E4521BD
:1028D000036E01C0E9FFEA6EEF50200819E10D0E0A
:1028E00044250201256F000E010145210201266FDA
:1028F000286F25C227F20001CAEC04F001C034F1B0
:102900000101345305E0342D01D002D0010E346FA3
:102910007AD345C128F244C127F2010E02012A6F81
:10292000B30E296F0A0E2B6F00015CEC04F001520C
:1029300039E10A0E01014425016E000E4521036EA6
:1029400001C0E9FFEA6EEF520EE135C126F21F0E1B
:102950000201276F0001B1EC05F0010135519EA87D
:10296000FED7AD6E1ED00A0E4425016E000E452125
:10297000036E01C0E9FFEA6EEF50200812E10B0E72
:1029800044250201256F000E010145210201266F39
:10299000286F25C227F20001CAEC04F001C035F10E
:1029A000010131D345C128F244C127F2010E0201D1
:1029B0002A6FBE0E296F050E2B6F00015CEC04F030
:1029C00001520EE101013753D8A402D0000108D012
:1029D00096908D90E60E006E002EFED7968013D353
:1029E00045C128F244C127F2010E02012A6FC40E2C
:1029F000296F050E2B6F00015CEC04F001522FE1F2
:102A000001013753D8A402D0000129D043530CE16F
:102A100029C125F2000175EC0AF00152D8B402D0A8
:102A2000010102D0000E01D0010E0101436F110E11
:102A30001E6E435310E10201936B1E0E926F010E46
:102A4000946F000105EC04F00152D8B402D00101EA
:102A500002D0000E01D0010E0101436FD4D245C156
:102A600028F244C127F2010E02012A6FCA0E296F13
:102A7000050E2B6F00015CEC04F001522FE1010107
:102A80003753D8A402D0000129D043530CE129C107
:102A900025F2000175EC0AF00152D8B402D0010110
:102AA00002D0000E01D0010E0101436F010E1E6E17
:102AB000435310E10201936B1E0E926F010E946F4F
:102AC000000105EC04F00152D8B402D0010102D09B
:102AD000000E01D0010E0101436F95D245C128F2CD
:102AE00044C127F2010E02012A6FD00E296F050E94
:102AF0002B6F00015CEC04F0015244E101013753FB
:102B0000D8B402D000013ED0050E4425016E000E5F
:102B10004521036E01C0E9FFEA6EEF520EE136C1B6
:102B200026F21F0E0201276F0001B1EC05F0010132
:102B300035519EA8FED7AD6E24D0050E4425016EFA
:102B4000000E4521036E01C0E9FFEA6EEF50200838
:102B500018E1060E44250201256F000E01014521F2
:102B60000201266F286F25C227F20001CAEC04F08B
:102B700001C036F10101365304E0362D01D001D0F9
:102B8000366B41D245C128F244C127F2010E020141
:102B90002A6FD60E296F060E2B6F00015CEC04F035
:102BA00001524CE1060E01014425016E000E452143
:102BB000036E01C0E9FFEA6EEF520EE137C126F263
:102BC0001F0E0201276F0001B1EC05F00101355124
:102BD0009EA8FED7AD6E31D0060E4425016E000EC4
:102BE0004521036E01C0E9FFEA6EEF50200825E1A0
:102BF000070E44250201256F000E01014521020147
:102C0000266F286F25C227F20001CAEC04F001C02C
:102C100037F10101375305E0372D01D002D0010E05
:102C2000376F0001E0EC01F00101375306E00201CB
:102C3000256B000113EC04F00101E5D145C128F238
:102C400044C127F2010E02012A6FF10E296F090E0D
:102C50002B6F00015CEC04F00152D8A4F9D0090EEE
:102C600001014425016E000E4521036E01C0E9FFFC
:102C7000EA6EEF520EE138C126F21F0E0201276FF5
:102C80000001B1EC05F0010135519EA8FED7AD6EF3
:102C9000DED0090E4425016E000E4521036E01C0F1
:102CA000E9FFEA6EEF502008D8A4D1D00A0E4425DF
:102CB0000201256F000E010145210201266F286FD8
:102CC00025C227F20001CAEC04F001C038F101016D
:102CD000385305E0382D01D002D0010E386F382D61
:102CE000B6D0010EA96E37C1A8FFA69CA69EA684E9
:102CF000F2CF00F0F29E0F01550EA76EAA0EA76E3E
:102D0000A682A6B2FED7A6940050F212020EA96EB9
:102D100029C1A8FFA69CA69EA684F2CF00F0F29E31
:102D2000550EA76EAA0EA76EA682A6B2FED7A694CF
:102D30000050F212030EA96E35C1A8FFA69CA69EF4
:102D4000A684F2CF00F0F29E550EA76EAA0EA76ED3
:102D5000A682A6B2FED7A6940050F212040EA96E67
:102D600034C1A8FFA69CA69EA684F2CF00F0F29ED6
:102D7000550EA76EAA0EA76EA682A6B2FED7A6947F
:102D80000050F212050EA96E2FC1A8FFA69CA69EA8
:102D9000A684F2CF00F0F29E550EA76EAA0EA76E83
:102DA000A682A6B2FED7A6940050F212060EA96E15
:102DB00030C1A8FFA69CA69EA684F2CF00F0F29E8A
:102DC000550EA76EAA0EA76EA682A6B2FED7A6942F
:102DD0000050F212070EA96E33C1A8FFA69CA69E52
:102DE000A684F2CF00F0F29E550EA76EAA0EA76E33
:102DF000A682A6B2FED7A6940050F212080EA96EC3
:102E000036C1A8FFA69CA69EA684F2CF00F0F29E33
:102E1000550EA76EAA0EA76EA682A6B2FED7A694DE
:102E20000050F212090EA96E38C1A8FFA69CA69EFA
:102E3000A684F2CF00F0F29E550EA76EAA0EA76EE2
:102E4000A682A6B2FED7A6940050F2120101DBD0F2
:102E500045C128F244C127F2020E02012A6F030E77
:102E6000296F050E2B6F00015CEC04F0015219E193
:102E700001013753D8A402D0000113D00001BEEFE6
:102E80000AF001C025F201C026F21F0E0201276FD1
:102E90000001B1EC05F0010135519EA8FED7AD6EE1
:102EA000B2D045C128F244C127F2010E02012A6FB7
:102EB000FB0E296F070E2B6F00015CEC04F0015232
:102EC0003BE101013753D8A402D0000135D0070EF1
:102ED0004425016E000E4521036E01C0E9FFEA6E34
:102EE000EF5207E129C127F20001C9EC0AF022D014
:102EF0000101070E4425016E000E4521036E01C03D
:102F0000E9FFEA6EEF50200816E1080E44250201A1
:102F1000256F000E010145210201266F286F25C291
:102F200027F20001CAEC04F001C026F201C027F22A
:102F3000C9EC0AF0010167D045C128F244C127F26B
:102F4000020E02012A6F090E296F080E2B6F000175
:102F50005CEC04F001523FE101013753D8B402D0D8
:102F6000000139D0080E4425016E000E4521036E84
:102F700001C0E9FFEA6EEF520EE139C125F21B0EE6
:102F80000201266F000124EF0BF0010135519EA8CC
:102F9000FED7AD6E1ED0080E4425016E000E4521F1
:102FA000036E01C0E9FFEA6EEF50200812E1090E3E
:102FB00044250201256F000E010145210201266F03
:102FC000286F25C227F20001CAEC04F001C039F1D4
:102FD000010119D000010101312D15D00201256B2D
:102FE0002551000176EC01F00201252B006E005006
:102FF0009EA8FED7AD6E150E255DF2E1010135519B
:103000009EA8FED7AD6E000199D00101375329E08B
:1030100043530CE129C125F2000175EC0AF001527D
:10302000D8B402D0010102D0000E01D0010E01017E
:10303000436F400E2A251E6E435310E10201936B2D
:103040001E0E926F010E946F000105EC04F0015208
:10305000D8B402D0010102D0000E01D0010E01014E
:10306000436F375302E142A141D02F51030827E0BB
:10307000435311E145C126F244C125F20201276BF9
:10308000286B000166EC0BF00152D8B402D00101AC
:1030900002D0000E01D0010E0101436F43530EE137
:1030A000010E0201266F2C0E256F276B30C128F20E
:1030B000000166EC0BF001C043F1010117D043534E
:1030C00012E145C126F244C125F20201276B010E2F
:1030D000286F000166EC0BF00152D8B402D0010158
:1030E00002D0000E01D0010E0101436F335325E0E1
:1030F000375323E045C126F244C125F23F0E0201B9
:10310000276F000175EF0BF002C026F201C025F217
:103110000201255302E126530CE001014353D8B4C8
:1031200002D0020106D030C125F20001C3EC08F044
:1031300005D00101435301E0436B00010101375306
:10314000D8A492D0928280B26AD0928280B266D0A5
:10315000929A899A0201936B1E0E926F000110ECF5
:1031600008F092988988400E010129251E5C02E131
:10317000428152D0200E29251E5C02E142834CD0B0
:103180001E503F0802E1429347D01E505F0802E103
:10319000429142D01E50180802E142853DD01E5097
:1031A000190802E1429538D01E5014080DE1140EA2
:1031B0009EA8FED7AD6E35519EA8FED7AD6E429348
:1031C00042914295396B28D01E5011080BE142A361
:1031D00009D0110E9EA8FED7AD6E35519EA8FED720
:1031E000AD6E1AD01E2C0BD042A309D0010E9EA8A2
:1031F000FED7AD6E35519EA8FED7AD6E0DD01E50D8
:1032000008080AE142A308D0080E9EA8FED7AD6EBA
:1032100035519EA8FED7AD6E929A898A25D00F0EA1
:10322000006E002EFED7928280A21ED042A30AD04A
:10323000929A899A30C125F20001C3EC08F001018D
:10324000429312D042A110D042A50ED0010E02012D
:10325000266F390E256F010E276F286B000166EC73
:103260000BF001014295429100010CEF0FF00300B9
:020000040030CA
:0E00000000021E19008381000FC00FE00F40A8
:00000001FF
